:1000000000308A007828000083160515003083121E
:1000100005190130F700770DAB00AB0DAB0DF830D3
:10002000AB05831685150030831285190130F70062
:10003000F70DF70DFC30F70577082B07AD00831699
:10004000051600308312051A0130F7000310F70D72
:1000500077082D07AF0083160614003083120618A8
:1000600001302F07A4008A118C28AC012C08073C12
:10007000031C61282C08073CAD002B08F7002D0855
:10008000F800031947280310F70CF80B4328771CD6
:100090004E2883160612831206165228831606125D
:1000A0008312061283168612831286160330F70017
:1000B000F70B58285B288316861283128612AC0A27
:1000C000362800342A308400831300080319762868
:1000D0000330F800F701F70B6B28F80B6A283C3067
:1000E000F700F70B71287428800B68288A112929DA
:1000F000840183131F3083058316851183128515B0
:1001000007309F008316851083128514A9012908E2
:10011000093C031C2B290428240DF700F70DF70DCB
:10012000F830F7057708AA002130AB002A088316BB
:100130009B009C131C141A088312A300240DF700C3
:10014000F70DF70DF830F7057708013EAA002130CA
:10015000AB000318AB0A2A0883169B009C131C14DF
:100160001A088312A200240DF700F70DF70DF830DE
:10017000F7057708023EAA002130AB000318AB0A4E
:100180002A0883169B009C131C141A088312A100D2
:10019000240DF700F70DF70DF830F7057708033E4B
:1001A000AA002130AB000318AB0A2A0883169B0073
:1001B0009C131C141A088312A0002308A80022080C
:1001C000A7002108A6002008A500831605108312A9
:1001D00005140830F700F70BEB288316051083127F
:1001E000051083160513831205170830F700F70B67
:1001F000F72883160513831205130130AB00352051
:10020000AB013520AB0135206030AB003520043028
:10021000AB0035202808AA00AB0035202708AA002B
:10022000AB0035202608AA00AB0035202508AA001F
:10023000AB00352083168611831286150830F7002F
:10024000F70B202983168611831286113230AA00FB
:100250006228A90A872883168510831285106300F7
:02026000630039
:084200000A00AA00AA00CE008A
:084210000A00AA00AB005D00EA
:084220000A00AA00AC00100026
:084230000A00AA00B800A50075
:0842400015005500550079003E
:0842500015005500560008009E
:08426000150055005600BB00DB
:08427000150055006300500029
:084280001500D200F100CD0091
:084290001500D200F2005C00F1
:0842A0001500D200F3000F002D
:0842B0001500D200FF00A5007B
:0842C0001C009600EB00D20087
:0842D0001C009600EC006100E7
:0842E0001C009600ED00140023
:0842F0001C009600F900A90072
:02400E00633F0E
:00000001FF
